:1000000001308A0021290000031787018801890136
:1000100083160908C039890003131F129F1201308B
:1000200003178800831203131F179F1783169F1748
:1000300083121F149412A1122108831687008312C1
:1000400021162108831687008312A1112108831627
:100050008700013083129400003083169400093029
:100060008312031785000F30F700031381018130DD
:10007000840083130008C03907388000640000083A
:10008000C739F719C0397704800035309000003047
:10009000F800920000308316920083122115210887
:1000A000831687008312970183169B019C01013000
:1000B0009D008312A11421088316870083129D01DD
:1000C0009412A11221088316870083122116210899
:1000D000831687008312A11121088316870001303F
:1000E00083129400003083169400093083120317A2
:1000F00085000F30F70003138101813084008313E2
:100100000008F0390738800064000008F739F71953
:10011000F039770480008A110A124929AC010408D9
:10012000AB002C10831B2C14A51F9E28AB172B1E75
:10013000AB0AA409A509A40A0319A50A250EF038DB
:10014000A700A707E23EA800323EAA0025080F3903
:10015000A807A807AA07E93EA900A907A907240E2E
:100160000F39A907AA07A90DAA0DAA09AA0D2408E3
:100170000F39AA07A70D0730A6000A30AA07A9035E
:10018000031CBE28A907A803031CC228A807A703AD
:10019000031CC628A707A603031CCA282630840010
:1001A000831307302B052B1384032B05031DDF2836
:1001B0002B1A840A2B1ADF282030F700FC2884072A
:1001C0002A30040203192B170008F700031DF0283A
:1001D0002B1BF0282B1A0129AB19F0282030FB2803
:1001E000AB1FF8282D30F70084032B13AB13FC282A
:1001F000AB152B123030F707770864000C1EFD2872
:100200009900840A2B1FE0288A110A125C292330E6
:1002100084008313000803191E290230F800BF3040
:10022000F7006400F70B1129F80B0F299630F7003F
:10023000F70B18291B296400800B0D298A110A125B
:100240006629840183131F308305713083168F0064
:100250000F088312A0018316031787110C300313B4
:100260009900A2309800903083129800FF30A100CE
:10027000831603170908C039890003131F129F1240
:100280000030031788008312870188018901031356
:10029000042864009F149F184B291E08FA00831637
:1002A0001E088312A2001E08A3000B3084001E0843
:1002B000A5002208A4008E281A3064000C1E5D29B7
:1002C00099000430A200FA30A3000729A20B632989
:0402D0004929630055
:04400E008C2FFF3FB5
:00000001FF
